:020000041000EA
:1000000000B5324B212058609868022188439860DF
:10001000D860186158612E4B002199600221596106
:100020000121F02299502B49196001219960352056
:1000300000F044F80222904214D00621196600F024
:1000400034F8196E01211966002018661A6600F04E
:100050002CF8196E196E196E052000F02FF8012189
:100060000842F9D1002199601B49196000215960AB
:100070001A491B48016001219960EB211966A021F2
:10008000196600F012F800219960164914480160C1
:100090000121996001BC002800D000471248134993
:1000A000086003C880F30888084703B5996A0420EC
:1000B0000142FBD001200142F8D103BD02B5186610
:1000C0001866FFF7F2FF186E186E02BD00000240BE
:1000D000000000180000070000035F00212200005C
:1000E000F4000018222000A00001001008ED00E03C
:1000F00000000000000000000000000074B24E7A12
:1001000000200420F7010010CB010010CD010010E9
:10011000C9010010C9010010C9010010C901001077
:10012000C9010010C9010010C9010010CF01001061
:10013000C9010010C9010010D1010010D301001045
:10014000C1010010C1010010C1010010C101001067
:10015000C1010010C1010010C1010010C101001057
:10016000C1010010C1010010C1010010C101001047
:10017000C1010010C1010010C1010010C101001037
:10018000C1010010C1010010C1010010C101001027
:10019000C1010010C1010010C1010010C101001017
:1001A000C1010010C1010010C1010010C101001007
:1001B000C1010010C1010010C1010010C1010010F7
:1001C000EFF30580103800BE00BE00BE00BE00BECA
:1001D00000BE00BEF2EB8871844F0010A44F0010E7
:1001E0003802001090A31AE71E481F49086006C88D
:1001F00081F3088810471D480068002801D019487D
:10020000F3E70DA40ECC002902D000F012F8F9E7B4
:100210001749184A002000E001C19142FCD116495B
:100220008847164988471649884700BEFDE701C937
:1002300001C29A42FBD37047A44F0010C0000020B7
:1002400008160020EC6400100000042000000420C8
:10025000EC640010001004200010042000000000D6
:10026000704700000000000008ED00E0000000D032
:1002700008160020A8240020012200103D090010CB
:10028000F9210010F8B5C0460448054B10B583426B
:1002900003D0044B002B00D0984710BD0816002057
:1002A000081600200000000006480749091A8B10B4
:1002B000C90FC91810B5491003D0044B002B00D04A
:1002C000984710BD08160020081600200000000006
:1002D00010B5074C2378002B09D1FFF7D5FF054B4C
:1002E000002B02D0044800E000BF0123237010BDA2
:1002F000881900200000000098470010054B10B539
:10030000002B03D00449054800E000BFFFF7CCFFF5
:1003100010BDC046000000008C1900209847001056
:100320000300093BDBB2752B03D81F4A9B00D3584F
:100330009F46002070475D38C0B2FBE73D38C0B231
:10034000F8E71338C0B2F5E73120F3E73320F1E7DF
:100350002E20EFE73820EDE73720EBE73520E9E7FF
:100360002F20E7E73020E5E73420E3E72D20E1E721
:100370003620DFE72720DDE72620DBE72420D9E74A
:100380002520D7E72820D5E72220D3E72320D1E76F
:100390001E20CFE72120CDE72020CBE72B20C9E787
:1003A0001F20C7E72C20C5E7CC4A0010F0B5CE4689
:1003B0004746050080B5534B83B028000024E9462A
:1003C000984603F071FBA0420BD92F5D3800FFF770
:1003D000A7FF061E0AD10134280003F065FBA042E6
:1003E000F3D803B0C0BCB946B046F0BD0622002128
:1003F000484601F0B9FE4B461E703B00413B192BAD
:100400007DD93900404603F091FB431E98414700D7
:1004100004E001200021404202F09EFA002003F097
:1004200017F80028F5D04B463A000121002003F0D0
:100430002BF801F0B5F800295BD0FA2200239200D6
:1004400001F0B6FB07000BE0FA220023920001F056
:10045000AFFB874218D101200021404202F07CFA14
:1004600001F09EF80029EFD1FA21890001F062FB2A
:10047000B842F0D0002002F0EBFF002809D10120A3
:100480000021404202F068FA002002F0E1FF00285B
:10049000F5D0002300220121002002F0F5FF01F039
:1004A0007FF800291FD0FA220023920001F080FB80
:1004B00007000CE0FA220023920001F079FB87424A
:1004C00000D088E701200021404202F045FA01F007
:1004D00067F80029EED1FA21890001F02BFBB84220
:1004E000F0D0013478E7FA21890001F023FB0700FE
:1004F000EDE7FA21890001F01DFB0700B0E70227B4
:100500008CE7C04698470010F0B5DE464E46574689
:100510004546E0B585B003F0FFFA8146002847D094
:100520000622002102A801F01FFEA64F484639000E
:1005300003F0E8FA041E38D0002300269B46A24BA5
:10054000A24D9846A24B9A46A24B009323782200D4
:100550000320002B09D0E95C0140012900D197E07C
:10056000137053780132002BF5D14146200003F07F
:10057000F3FF002800D199E05146200003F0ECFF82
:10058000002800D192E02000009903F0E5FF002848
:1005900000D08EE004231E433900002003F0B2FA9D
:1005A000041ED3D15B4633430ED1484601F0C4FD4F
:1005B00005B0F0BCBB46B246A946A046F0BD01203E
:1005C0000021404202F0C8F9002002F041FF00285B
:1005D000F5D03200012102AB002002F055FF00F0FF
:1005E000DFFF002900D1ADE0FA220023920001F0E4
:1005F000DFFA04000BE0FA220023920001F0D8FA9F
:10060000844218D101200021404202F0A5F900F0F7
:10061000C7FF0029EFD1FA21890001F08BFAA0422F
:10062000F0D0002002F014FF002809D101200021A1
:10063000404202F091F9002002F00AFF0028F5D0B4
:10064000002300220121002002F01EFF00F0A8FF7D
:10065000002971D0FA220023920001F0A9FA0400C7
:100660000BE0FA220023920001F0A2FA84429CD10E
:1006700001200021404202F06FF900F091FF0029B3
:10068000EFD1FA21890001F055FAA042F0D08CE7B1
:100690002033137053780132002B00D05BE74146C2
:1006A000200003F059FF002800D065E701231E4316
:1006B00072E72000484903F04FFF002802D10223CF
:1006C0001E4369E72000454903F046FF002802D198
:1006D00008231E4360E72000414903F03DFF002846
:1006E000F6D020003F4903F037FF0028F0D020006B
:1006F0003D4903F031FF00282AD020003B4903F098
:100700002BFF002824D02000394903F025FF0028C2
:1007100052D02000374903F01FFF002805D023786E
:10072000222B2ED16278002A2BD15B46052B00D9D3
:1007300032E73422013310E0FA21890001F0FAF99E
:1007400004009AE7FA21890001F0F4F904005EE759
:100750005B46052B07D84C220133584602A9DBB271
:100760009B460A5418E72000224903F0F5FE0028B2
:1007700000D111E72378222B03D16278002A00D11F
:100780000AE7272B02D16378002BCED0200003F09C
:100790008BF9012800D0FFE65B46052B00D9FBE66C
:1007A0000133DBB220780193FFF7BAFD5946019B74
:1007B00002AA9B465054EFE65B46052BD3D828226D
:1007C0000133CAE7B0470010B4470010814E001053
:1007D000BC470010C4470010C8470010D0470010A5
:1007E000D4470010D8470010DC470010E047001045
:1007F000E8470010F047001070B500F0D1FE002966
:1008000000D17DE0FA220023920001F0D1F904002A
:100810000DE0FA220023920001F0CAF93B4B001BC5
:10082000984210D801200021404202F095F800F0D3
:10083000B7FE0029EDD1FA21890001F07BF9334B95
:10084000001B9842EED93248FFF75EFE00F0A8FE8A
:1008500000294FD0FA220023920001F0A9F90400E8
:10086000FA25AD000CE0FA220023920001F0A0F975
:10087000001BA8420FD201200021404202F06CF878
:1008800000F08EFE0029EED1FA21890001F052F924
:10089000001BA842EFD31F48FFF788FD1E48FFF753
:1008A00085FD1E4C2000FFF781FD1D48FFF77EFDF2
:1008B0002000FFF77BFD1B48FFF778FD2000FFF7C6
:1008C00075FD1948FFF772FD2000FFF76FFD17480F
:1008D000FFF76CFD2000FFF769FD1548FFF766FD87
:1008E0002000FFF763FD1348FFF760FD0122124B64
:1008F0001A7070BDFA21890001F01CF90400AFE7FD
:10090000FA21890001F016F9040090E7B70B000006
:10091000F8470010044800100C4800102848001048
:100920003048001060480010A0480010E448001053
:100930003049001078490010A524002010B501F0BE
:1009400053FD0021002002F049FF084C0120002146
:10095000404202F001F8002002F07AFD0028F5D0B4
:100960002378002BF2D1FFF747FFEFE7A524002003
:10097000002070477047C04600487047DC4C0010AC
:1009800000487047B84C001000487047A44C001055
:1009900070B5002823D003282CD8174B8000C558E9
:1009A000280003F081F8C0B2041C1F2812D8E4B25A
:1009B000002808D00023114AE95C01331180D9B224
:1009C00002328C42F8D8C0220134E3B25B009200BC
:1009D00013430CE01F24E4B20028EBD1F3E7064BED
:1009E00002221968054801F0C5FBC1239B00044899
:1009F000038070BD0020FCE7E00F0020061D0020F2
:100A0000041D00208023DB051868000F7047C046D6
:100A10000FB400B5084883B001F034FD049B002BEF
:100A200007D005A91800019101F0B2FB034801F0BD
:100A300029FD012001F0C4FBC4490010D449001075
:100A400070B5EFF3108C72B60D4D2B68002BFCD0F7
:100A5000BFF35F8F0724CB08C618C05C01230C408E
:100A6000A3401C000440034207D118433070BFF379
:100A70005F8F2C608CF3108870BD1000FFF7C8FFEB
:100A80002C0100D0F8B54746CE46884680B5EFF336
:100A9000108C72B61C4D2C68002CFCD0BFF35F8FFD
:100AA0009A4222D807210126894602E00132934268
:100AB00018D34D4637001540AF40D4080119045DE6
:100AC0002742F3D110003C430C70BFF35F8F00222C
:100AD0000D4B1A608CF3108800280EDBC0BCB946A1
:100AE000B046F8BD01204042EFE7BFF35F8F00231F
:100AF0002B608CF31088012040424346002BEDD040
:100B00000898FFF785FFC0462C0100D0044A1078F2
:100B1000431CDBB2172B00D9102313707047C0465B
:100B2000F00F002010B5064B064C82B00100009378
:100B300018221F232000FFF7A5FF02B010BDC046FA
:100B4000D8490010382000200021044B044ABFF38C
:100B50005F8F02C39342FAD17047C046000100D0B4
:100B6000800100D0054B064A1360064A13605360AB
:100B70009360D3601361536193617047808080807C
:100B800000E400E004E400E01F2318401E3B834023
:100B9000002905D0C021044A490053501360704712
:100BA000802201498B50FAE700E100E070B50D00AA
:100BB000EFF3108672B60F4A1368002BFCD0BFF318
:100BC0005F8F0D4B10309B6884001B590B4A93427A
:100BD00003D09D4201D000F083FE074B9B681D515E
:100BE000BFF35F8FBFF35F8F0022024B1A6086F363
:100BF000108870BD240100D000ED00E0C10100109C
:100C0000F0B557464E46DE464546E0B585B006008F
:100C100000911700EFF3108B72B66A4A1368002B2D
:100C2000FCD0BFF35F8F0025674B5D579A46002DC0
:100C300000DAA9E06B00654C01935B199B009846B4
:100C4000A146C1444B4652469B7910361370604B07
:100C5000B6009B6899590B1B2F2B33D95D4B9942DA
:100C600000D0ACE0019B42469C465B4B6544AD0026
:100C700063535A4B0232A218043B9B1A1B05584A75
:100C80005B0D651913436B80564B0121AB80FF232D
:100C9000AB71009BEF71AB604B460B4319004C4BA3
:100CA0009B689951BFF35F8FBFF35F8F0022454B65
:100CB0001A608BF3108805B0F0BCBB46B246A9465B
:100CC000A046F0BD01200A008243D3798C46BB4286
:100CD00031D84546130044491B1B5B415943090D5C
:100CE0003D4B63533D4B02356519043B5B1B1B05B4
:100CF0003B4D5B0D2B43AA464D466B800425AC460D
:100D00005546E044131F44441B1B1B055B0D1D434C
:100D10004B46997100999D8099604946DF71334B2C
:100D200001431360BBE75800C01880002018C17948
:100D3000B9422FD902000623D356002BF3DA0293CF
:100D40002B4B61460393131D9A4604235B429C463A
:100D5000E14450464B461B1A1B055B0D9C46204B3D
:100D6000957198466346404603439380019B5A1908
:100D70009200039BA418A380029B1C4AA371009BB2
:100D80002260E771A3608AE700F0AAFD00255346C0
:100D90005D574FE7908802934005131D9A4603154F
:100DA00061469C464046D444634604302018181AD5
:100DB000E0230005400D1B0218430390C5E700F037
:100DC0008FFD4FE7240100D0A4240020F40F002061
:100DD00000ED00E0C101001000A1FFFF2410002081
:100DE00000E0FFFF01BDFFFFAAAA00000148804705
:100DF00001BD000070B501240443EFF30581EFF35A
:100E0000108C72B6214A1368002BFCD0BFF35F8FA1
:100E10001F4B05001F4AED1A6D416A43120D1E4D0E
:100E20008900AE6852B27658A6421CD006215956A7
:100E300091421CD012215956914222D01E2159565E
:100E4000914220D02A2159560324914210D0134BAD
:100E500019781A708171BFF35F8F00220B4B1A60F3
:100E60008CF3108870BDAB680D4C5C50EFE700242C
:100E70006100091989005B18FF219971094999805E
:100E8000E5E70124F4E70224F2E7C046240100D09C
:100E9000F40F0020AAAA000000ED00E0A424002026
:100EA000C101001001BDFFFF024B9C466144890057
:100EB000016070474000003470B5114C114DAC42D8
:100EC0000FD2FF262368002B0CD0FFF71FFE010076
:100ED0002000FFF7E9FFA680BFF35F8F0834AC4224
:100EE000F0D370BDFFF712FE01002000FFF7DCFF1A
:100EF0002671BFF35F8F0834AC42E3D3F1E7C046FD
:100F0000F81500200816002010B50400FFF7FEFDBC
:100F100001002000FFF7C8FFFF232371BFF35F8F9D
:100F200010BDC04610B504000120FFF7FBFD034BC8
:100F3000C3189B002360BFF35F8F10BD40000034D7
:100F40000A4B1968EFF3108072B60A68002AFCD0C9
:100F5000BFF35F8F1B68BFF35F8F00221A6080F3BF
:100F6000108840BF002000217047C0469C2400200C
:100F7000F0B5DE4657464E464546E0B587B0EFF33E
:100F80000583032201251A40954091008846A94611
:100F9000B34B03925C58B34B1D60B34B04934B4669
:100FA000B24843630823E55E002D37DAA3881BB2FD
:100FB000002B00DBADE0A379002B00D0EEE008238E
:100FC000E05E002820DB430062691B18DB00D318B9
:100FD0009E68DD68731C00D111E1A4480100414402
:100FE000826A0B69B71A9B1A9F4215D30123026AC2
:100FF000039883401A420FD09C4800F0C9FA8D42F2
:1010000002DCCCD18642CAD940BF07B0F0BCBB4697
:10101000B246A946A046F0BD0E61EDE762696B00DD
:1010200092465B19DB009A4453469E68DF6800F0E5
:10103000AFFA8F42BADC00D103E1002F00DAE8E01A
:101040005246534652691B699346049A934200D113
:10105000D9E052460821605E528800045946104388
:101060009847009001910099019A0B0010001343DA
:1010700000D1CEE013000A00B61A9F41002806DB1B
:101080007A4800F085FA009E019F36184F4153467A
:101090009E60DF6000229A5E002A00DA86E7530035
:1010A00099186069C900411802938B68C9689B460A
:1010B000B94200DD7AE702D1B34200D976E70823CE
:1010C0009C46A444059565462281A446029B2C00BB
:1010D00006E053009918C90041188D68C968AB46ED
:1010E0009B18DB00C318B94206DC00D1B3E01C003A
:1010F0000023E25E002AECDA230064469C46534655
:101100001A806346059D1D80A3881BB2002B00DA60
:1011100051E72269EFF3108172B61368002BFCD0FF
:10112000BFF35F8F0123A7885B42A3803FB223698F
:10113000BFF35F8F00221A6081F31088002F00DA5E
:1011400039E72300083322009A4666697B00DB19E1
:10115000DB00F318996850468C460824115FDD685F
:10116000002910DB029306E0AB4244D00023E15E8D
:101170002000002906DB4C006418E4003419E36801
:10118000AB42F1DD029B078000201F5E1980002F1B
:10119000DCDA1400A379002B00D110E70023A3713F
:1011A00026000823E15E08364B1C00D12CE708001E
:1011B000A246656902E03E004B1C1AD04B005B184A
:1011C000DB00EF180A008C46E95E7B881BB2002B1F
:1011D000F1DA01235B42DC17BB60FC60824205D080
:1011E000534631801B893B8053461A8160464B1C15
:1011F000E4D15446E5E6A3686345B7D9C2E76B1C62
:1012000000D0EAE6F8E65B4658461B699847002896
:101210001BD153461B8822692381EFF3108372B6DA
:1012200011680029FCD0BFF35F8F514662880A80A5
:1012300022696580BFF35F8F0021116083F31088FE
:10124000B4E6864200D8F8E6B0E65B461A685B680A
:101250000092019307E7B34500D848E74CE7C04642
:10126000802400203C700540710F001000400540B4
:1012700070B52E4C2569002D04D00A212C48FFF7AB
:1012800013FE70BD2B4E0321300000F077F9E660AD
:10129000FFF73CFC284B03229C46D02322701B0600
:1012A0001B6801216370254B6044A3600F238000FD
:1012B00020610220638063694942A1801980023164
:1012C000198647311D83585218315A5275325C398C
:1012D000995218320131995218320131995218320B
:1012E00001319952083518329D5202311832995203
:1012F00018320131995218320131995218320131A4
:1013000099521832013199521832013199520C4BCD
:101310000C49DC6001303562FFF748FC01210320F5
:10132000FFF732FC084B1D60A7E7C0463C100020C9
:101330009C2400200040054040000034FFFF1000C6
:1013400080240020710F00103860054070B5010046
:101350000469EFF3108C72B620680028FCD0BFF34C
:101360005F8F02200D5E4C6968004019C000241890
:101370000869002D36DB26884E80BFF35F8F00267C
:1013800006608CF31088E360638804980133206161
:101390005B0405985B0CA26060611A1C002B1FD0D7
:1013A00093B22804628018430A69EFF3108C72B676
:1013B0001368002BFCD0BFF35F8F8B8823808D8058
:1013C0000B69BFF35F8F00221A608CF310880B78D3
:1013D00001329A40CB6808498C4663441A6070BD5C
:1013E0000122DDE7BFF35F8F002303608CF31088D9
:1013F00001204042F3E7C0463C20000010B543897D
:101400000A1493421ADD53009B184269DB00D3187B
:101410000469EFF3108C72B62268002AFCD0BFF387
:101420005F8F5A88090494B2090C8A4208D0036974
:10143000BFF35F8F00221A608CF31088002010BD6C
:101440008022120214435C80012302698371BFF37E
:101450005F8F002111608CF31088044902788C465C
:101460009340C268012062441360E8E73C2000001A
:10147000F0B557464E46DE464546E0B506000F003D
:1014800085B0EFF3058399468B46002B12D038497F
:1014900000204B6ABB4206D38A6ADB1B591E8B4174
:1014A000B2424041184305B0F0BCBB46B246A94623
:1014B000A046F0BD2F4B9A46DB68984653461B78F2
:1014C0004046039300F064F84246039B0400043353
:1014D0009B009B580D001B1A39003000001BA941CE
:1014E000894510DC0DD020BF214A0020536A5B459E
:1014F000D9D3926ADB1B591E8B41B242404118433B
:10150000D1E78342EFD900F04BF832003B00121ACA
:101510008B41002B1ADB00230193174B3200009301
:1015200050463B00FFF712FF011E0FDD104B5A6AB9
:101530005A451BD39B6AB34216D35046FFF75EFF52
:101540000B4A0020536A5B45ADD3D2E7084A00201E
:10155000536A5B45A7D30020926ADB1BB24240412D
:101560005A1E934118439EE75A45E6D120BFE4E74F
:10157000004005403C100020410F001010B5024A09
:101580000248FFF75DFA10BDF44900103C2000202E
:101590000300416A0A00986A596A8A42FAD1704780
:1015A000034B596A0A00986A596A9142FAD1704706
:1015B00000400540F8B5DE464E4657464546E0B584
:1015C0008B4605000A991800160000F0B3FA0A9B32
:1015D0006C001F02324B64199C46A400644463688B
:1015E00081469F4200D967602B1FDBB29846012BD2
:1015F00030D9C02380229B01E31812011A60294BC5
:10160000AD0059599A4600291BD17301E026226882
:1016100053401E40802342465B01E3181E60012AAE
:1016200030D9802380229B01E31812011A605346AF
:101630004A4667605A51F0BCBB46B246A946A0462E
:10164000F8BD586900F076FA013043001B18033BDF
:10165000FDD2DAE75B46012BCBD1C02303229B01ED
:10166000E3181A60023AA3681A42FCD07301E0261C
:101670002268AD0053401E4080230A4A5B01924617
:10168000E3181E605A462168514003220A401A603E
:1016900001225B469A40A3681A42FCD0C1E7C046CB
:1016A0000080004040200020F0B546464F46D64618
:1016B000C0B51F00344B44009C462418A400644469
:1016C000636888461600FF2B02D880235B006360A6
:1016D000031FDBB29A46012B30D9C02380229B0125
:1016E000E31812011A60294B8500595999460029BF
:1016F0001BD17301E026226853401E4080235246CE
:101700005B01E3181E60012A30D9802380229B01EF
:10171000E31812011A6080235B0063604B465F513F
:10172000E0BCBA46B146A846F0BD586900F002FADE
:10173000013043001B18033BFDD2DAE74346012B7F
:10174000CBD1C02303229B01E3181A60023AA3689D
:101750001A42FCD07301E0262268850053401E40E7
:1017600080230A4A5B019146E3181E6042462168C5
:10177000514003220A401A60012342469340A26866
:101780001342FCD0C1E7C04600800040402000204A
:10179000014B8000C058704740200020F8B504007D
:1017A00021481E0017000D0000F0C4F901003800A8
:1017B00000F0C0F9069B36041B031E432368002B70
:1017C00020DB1A4B1A49E3185A1E934180229201DA
:1017D00094465B421B0B174A1B0363441360164A73
:1017E00013601F000A689743FBD1144B2560E21871
:1017F0002123A06013602368002BFCDA0823E66035
:101800001360F8BD3F2322681340AB42D9D1A368CF
:101810001B051B0D8342D4D1EE22E368D202134094
:10182000B342CED1EDE7C046001BB7000040FDBF7C
:1018300008C0004000E0004000F00040043000001C
:101840008023024A9B000B43D3627047008005400F
:10185000002310B50100988A1B8B984710BDC04625
:10186000162310B50100188802331B88984710BD55
:10187000F8B54746CE4680B50F1E18D014239946BA
:10188000043304000025012698464B461888434639
:1018900021681B88984701C4431E984101350640C2
:1018A000AF42F2D13000C0BCB946B046F8BD012607
:1018B000F8E7C046AA23064A1B0113608D235B008C
:1018C000D3600449044B19605368002BFCDA70475D
:1018D0000040024000B0FA00006002407047C0467D
:1018E00010B50148FFF794F8184A001070B5074D7D
:1018F000074EB54209D20024013E761BB60808CD3A
:10190000984723000134B342F9D170BD504700100D
:101910008C470010054B064A06491A60064A074BD9
:101920001A6010000B689843FBD1704700E000403C
:10193000BFCDFBFE08C00040FE7F3C0000F0004031
:10194000044BDB6C002B03D18022034BD2021A60C4
:101950007047C046000011504C201150044A054BFE
:101960001A60054A1368DB018033FBD17047C0461B
:10197000FFFFFF0100F0004008C000404022034B81
:101980009A675A671A67DA667047C04600F00140E6
:1019900010B5FFF7D9F810BDF8B52749274C284DE9
:1019A000641AA6103200302E00D93022280092008E
:1019B00000F0E0FBBC2C3BD830202F232C1964070F
:1019C000204A801BE40F9B1B052B16D93700002CE7
:1019D00002D0B300771CEA50001B33199B0041086A
:1019E000EB18C900C9181A605A6008339942FAD135
:1019F000012303421CD09843C619B300EA50731C5C
:101A00002F2E15D09B00EA50B31C2E2E10D09B0019
:101A1000EA50F31C2D2E0BD09B00EA50331D2C2EC8
:101A200006D09B00EA50731D2B2E01D09B00EA507C
:101A3000054B9D60F8BDC04600010010C0010010BC
:101A400000000020C101001000ED00E0002310B5EF
:101A5000294C82B0A367FFF72DFF0122274B1A60A4
:101A6000636C012BFCD10322254B1A60224A936B35
:101A7000012BFCD1013300930121224A2248043377
:101A8000FFF78CFE052301210093204A2048FFF731
:101A900085FE0022022104201E4BFFF705FE0022D6
:101AA000012105201C4BFFF7FFFD0022002107202C
:101AB0001A4BFFF7F9FD002200210820174BFFF712
:101AC000F3FD8023DB000093002200210920134B4B
:101AD000FFF770FD0022104B00210620FFF7E4FD08
:101AE0000420FFF755FE0E4900F024F80100002005
:101AF000FFF7A6FE02B010BD008000403CB00040E1
:101B000030B00040002F685900800240008C8647AA
:101B100000C00240001BB70040597307006CDC0294
:101B200040420F0001480421014B1847601000207B
:101B300071180010114A936F9B0813D210665166FA
:101B4000002905D0FFE7FFE7FFE7516F106F7047EF
:101B500004B5002801D00020C04302F0C1FD0021DF
:101B600004BDC046F0B5146E556E576F166FFFF783
:101B7000E5FF1466556657671667F0BD000000D094
:101B800094464A4A926F9208624601D228E0C046C3
:101B9000F0B5464E346E756E776F366F00F020F8F4
:101BA0009446424A14665566576716676246F0BD0A
:101BB00094463E4A926F9208624601D254E0C04673
:101BC000F0B53A4E346E756E776F366F00F04CF8A4
:101BD0009446364A14665566576716676246F0BDE6
:101BE000002B24DB11D000293EDA00B5C943404266
:101BF00000D1013100F038F8C943404200D1013131
:101C0000DB43524200D1013300BD002AEBD1002852
:101C100001D1002905D00020C90FC90701D1C04357
:101C2000410800B502F04CFD0022002300BD00B5C4
:101C300000290ADBDB43524200D1013300F014F8E3
:101C4000C943404200D1013100BDC943404200D1E7
:101C50000131DB43524200D1013300F005F8DB4390
:101C6000524200D1013300BD002923D1002B18D1ED
:101C7000002A0CD0BC460D4F38667A66002100233E
:101C8000FFE7FFE7FFE77A6F386F67467047002886
:101C900001D00748010000B502F012FD0022002328
:101CA00000BD02000B00002000217047000000D0A2
:101CB000FFFFFFFF002B00D0BFE0130C28D1002A4C
:101CC000E7D080B4114F39667A66FFE7FFE730B49A
:101CD000040C7B6F396F1B0423433B667A66FFE776
:101CE000FFE7FFE7C04684B27B6F3D6F1B042343D1
:101CF0003B667A66FFE7FFE7C04600232C042D0C05
:101D00007A6F386F00196941B0BC7047000000D08D
:101D1000F0B594460025140E01D112020835140FB7
:101D200001D112010435940F01D192000235D40F74
:101D300001D152000135D40B0134254F7C66254C6E
:101D40003C660E0C93B2FFE7FFE7FFE73C6F66438C
:101D5000360C7703BE467343DF0B5B04C01AB941F0
:101D6000130C7343DB18C91ACE086643360CB6440D
:101D700093B273431F0F1B01C01AB941130C734375
:101D80001F0B1B05C01AB941860D8F023E436643E7
:101D9000360C092D24DB520A7243801A7703460A57
:101DA0006643360C16235B1BDE40DF40BF196446DA
:101DB0006643821B7046043506330100D940A840B3
:101DC000C01900D30131A24206D20023F0BD0000A9
:101DD000000000D0FFFFFFFF121B0130F3D3F1E73B
:101DE00009277F1BFE406446A2B27243801A00D2CC
:101DF0000139220C7243130C1204821A99410B0010
:101E00007046043513370100F940A840801900D30B
:101E10000131002B02D1A2420AD2F0BD013000D321
:101E20000131121BFAD2013BF8D1A24200D2F0BD1F
:101E3000013000D30131121BF7E7F0B51C0C00D0C4
:101E400080E00CB400251C0A04D11B02160E33439B
:101E5000120208351C0B04D11B01160F334312016B
:101E600004359C0B04D19B00960F3343920002353E
:101E7000DC0B02D192185B4101351C0097186441BC
:101E80000134464F7C66464C3C660E0CFFE7FFE78C
:101E9000FFE7C0463C6F6643360C7703BE4697B2F9
:101EA0007743C01B00D20139C01B00D201399FB259
:101EB0007743C91BC91B170C77437E04FF0B801B9C
:101EC000B941CE086643360C0C2D33DBB644120BF9
:101ED0001F053A431B0B97B27743C01B00D2013951
:101EE0009FB27743C91B170C77433E043F0C801BFE
:101EF000B941860D8F023E43664329277F1BFE4072
:101F00000C3D7746AF40BF1930BCA2B2ABB27243B2
:101F10007343801A9941220C7243130C1204801AE5
:101F2000994102000B000137001BA941F9D2781E2C
:101F30000021F0BD0C277F1BFE4077467F0BAF4092
:101F4000FF19E0E700245D1C07D0144F7D66396659
:101F5000FFE7FFE7FFE7FFE73C6F95B29EB26543FF
:101F60006643401BB141150C1E0C654366433604A5
:101F70002F0C3E432D04401BB141994204D2020074
:101F80000B0020000021F0BD01D19042F7D3801A50
:101F9000994101349942F2D3F6E70000000000D0E5
:101FA000FFFFFFFF132370B51D78012D19D014DD3D
:101FB0001F48FFF755FC06001E48FFF751FC1E4C5A
:101FC00080223100200000F0D5F8022D2DD01B48D2
:101FD000FFF73EFC1A4B186070BD1A4B164CA364F9
:101FE000F5E7184B144C23606360A360E360236142
:101FF0006361A361E36123626362A362E3622363BB
:102000006363A363E36323646364A364E36423659A
:102010006365A365E36523666366A366E36623677A
:102020006367A367E367A364D1E7064BA364CEE7C6
:102030005344000053460000881700204C33000032
:10204000982400204920001007B5604601880A0A3C
:102050000230DF2AFAD1C9B2820804D3028840884C
:102060000004104300E00068014A5050039007BD8F
:102070008817002051434343C9188C46110C83B282
:102080004B4310B4040C614392B280B2504362439C
:102090001C041B0C001910BC59411304120CC0186D
:1020A0005141614470470000132310B512481C7859
:1020B000FFF7D6FB0100012C0AD003DD80220F4878
:1020C00000F058F80E48FFF7C3FB0E4B186010BD28
:1020D0000A4C5422200000F04DF80B4B6365A365B9
:1020E000E36523666366A366E36623676367A367A6
:1020F000E3672362E361E5E75346000088180020A8
:102100004C330000982400200D21001007B56046D4
:1021100001880A0A0230DF2AFAD1C9B2820804D340
:10212000028840880004104300E00068014A5050D3
:10213000039007BD8818002070B50400054D2800E5
:1021400002F0FEFA200002F0DFF9280002F0B0FAF7
:1021500070BDC046F815002001480421014B184706
:102160007010002071180010014B1B681847000008
:1021700070100020014B5B681847000070100020B1
:1021800010B5002800D110BD00F032F9FBE7C046C1
:1021900010B5094A0300146884B0002C08D001224D
:1021A00000910648524203A9A047012004B010BD87
:1021B00000F068F90020F9E7782400208121001060
:1021C00000BEFDE7094A03001068002805D0084951
:1021D000C3188B4207D81360704706480449C318D8
:1021E00010608B42F7D901204042F5E774200020AF
:1021F00000000420A824002010B5FFF7E1FFC0462E
:1022000070B5FFF773FB074D074EB54209D20024A6
:10221000013E761BB60808CD984723000134B3422F
:10222000F9D170BD8C47001098470010030010B51D
:10223000080011001B68984710BDC046F0B5C6469F
:1022400000B5437D07000C001600002B46D0002A85
:1022500017DD0B780A2B24D000239846012E13D0CB
:1022600001252900635C01350A2B26D0B542F8D13F
:10227000464509DCA419013C23780D3B5A425341E1
:102280003B7580BCB846F0BD4346E018A419F11A6E
:10229000013C3B68984723780D3B5A4253413B75BC
:1022A000EFE7037D002BD7D102210F483B68984709
:1022B000012EDFD001239846D2E7631E5B5C0D2B15
:1022C000D4D0884504DA4346C91AE0183B689847D9
:1022D000022105483B68A8469847C7E703681100F4
:1022E00020009847CDE7C046784D0010F0B5454630
:1022F000DE464E465746E0B583B091461C00804608
:102300000D00FFF74DF90023304A12184B41002B06
:1023100002DA01222E4B52422E4908008A4602F070
:10232000EFF907006B1C03D1404601F0BDFB05002F
:10233000002C27D0284E294B1C68002C18D04B4667
:10234000002B21D1264B994602E02469002C0FD0A6
:102350002368002BF9D04B461B68002B01D09C4210
:10236000F3D120002A004146B0472469002CEFD168
:10237000002F26D1280003B0F0BCBB46B246A946C8
:10238000A046F0BD174ED6E7154B99460A239B464B
:1023900002E02469002CEBD02368002BF9D04B46D7
:1023A0001B68002B01D0A342F3D12A004146200034
:1023B000B0476B465A462000DA71D91D0122B0475A
:1023C000E7E7504602F074F9D4E7C04640420F00F8
:1023D000FFFFFF7F001600203D2200106820002034
:1023E000702000202D22001010B500F069F810BDFB
:1023F000F0B5CE46474680B583B06B460600DD1D7E
:102400002870FFF7CDF80023194A12184B41002B12
:1024100002DA0122174B524217490800884602F09F
:102420006FF9164B81461C68002C14D0144F02E043
:102430002469002C0FD02368002BF9D03B68002BB7
:1024400001D09C42F4D1200001222900FFF7F6FEC2
:102450002469002CEFD14B46002B05D1300003B08E
:10246000C0BCB946B046F0BD404602F021F9F5E7E0
:1024700040420F00FFFFFF7F001600206820002071
:102480007020002070B5040001F00EFB0123010054
:10249000050001222000FFF729FF084B1C68002CD3
:1024A00006D06368002B05D098472469002CF8D12A
:1024B000280070BD2469002CF3D1F9E768200020C2
:1024C0000020704710B5024800F004F810BDC04667
:1024D0009024002010B588B004000D220021684629
:1024E000FFF742FE0D22002104A8FFF73DFE4B231B
:1024F0006A466846137004A90D2202F0C9F8152136
:10250000082220006944FFF735FE08B010BDC04620
:10251000F8B500F047F90C23194DFF22AB670520F1
:102520001849FEF76DFB184C402200212000FFF7F0
:102530001BFE4027002301262121144A66702783B1
:10254000A260136063545F31618445396354104A5B
:1025500010496360E2602787A1620B606362E262F8
:1025600002F0B6F880239B052E64EB6490230A4AA0
:102570000120EA508022094B5202DA64F8BDC046BD
:1025800000001150490500207820002084001050E0
:10259000000110508000105010D001000020115098
:1025A00010B501210520FEF7EFFA10BD10B500228D
:1025B0000021024800F016F910BDC0469820002006
:1025C000044B1970002904D080219023024A89020B
:1025D000D1507047A1240020002011500B785B06D9
:1025E00002D14B78052B00D070478A78014B1A60D6
:1025F000FAE7C04600001150F0B5C646C87800B5ED
:102600008007830F1800012B60D08F780A794B79EF
:102610007F213940FC091B024E001343334D321910
:102620005201AA18977001276740577000275B0571
:102630005B0DD7701383D076B846CA00012C32D018
:102640002B4FBC468F016244BC46AC446746BA601F
:1026500047461760002932D0264AC9009046624694
:10266000414451603F223F339343022837D02249EF
:1026700037190A687F01D3180B602049EF19FA60F7
:102680008B422ED836197601AD19EB7E1C499B067C
:102690004A4013438022120613436A6813600120E4
:1026A00080BCB846F0BD174FBC468F016244BC46A3
:1026B000AC446746BA6247461760002908D1002338
:1026C00064012C196360104BE360E8E70020E7E742
:1026D0000B4AC9009046624641445162C2E75B0022
:1026E000C5E7FFF7FDF8FA68CCE7C0467820002080
:1026F00084001050040010507C240020FF0F105064
:1027000000001050800010500001105010B501F072
:10271000DFFF10BD10B57F200C0020404000E40911
:10272000110000191A00034B4001C01800F05AF8BC
:10273000012010BD782000207F23180000B508403C
:1027400083B00B4204D14B424B41084A013393669C
:102750008022C9094000064B401840010021C018E2
:10276000120101F0E5FF03B000BDC046002011508A
:10277000782000207F22130010B50B400A4200D1C0
:1027800010BDC9095B005B1804485B01C018002339
:1027900000220349C37001F0CBFFF1E7782000204D
:1027A000FFF7FFFF80220A4B520410B51A60094B55
:1027B00009491A6010000B689843FBD18022002160
:1027C00052010648FFF7D0FC0922054B5A6710BD9D
:1027D00000E0004000F0004008C000400000105041
:1027E00000001150002310B5C3820133828283762A
:1027F0000161040001F094FF002804D0802190239F
:10280000074A8902D150200001F04AFF002802D077
:102810000123237710BD200001F07AFFFAE7C046BC
:1028200000201150002070477047C0467047C046D6
:102830000020704700207047002070477047C04656
:102840007047C0467047C0467047C046024B587834
:10285000431E9841C0B270471C1E0020024B1878DE
:102860004007C00F7047C0461C1E0020F0B5D6467A
:102870004F464646C0B52D4B07009A461B780E00C2
:10288000FF2B4DD100293ED0002154222848FFF7CC
:102890006BFC0022274C284B20001A70FEF734FBFB
:1028A000264B1C60264C2000143CFEF73BFB20000E
:1028B00001F0DAF8234B244D1C60244B002B04D08C
:1028C000280000E000BF224B1860224A00249146F5
:1028D0001F4A2B7890460EE043461B6862019B1806
:1028E000002B10D05B68002B0DD0984701342B785B
:1028F000E4B2A34209D3A342EED8E31A5B014B44EE
:102900005B68002BF1D100200BE05346310038000A
:102910001F70FFF7FDFD0028F5D03800FFF740FEDF
:102920000120E0BCBA46B146A846F0BD9C1000208C
:102930001C1E0020141E0020A2240020701E002057
:1029400094100020741E0020A0240020000000002D
:10295000AC1C0020244E0010F0B5DE4657464E4613
:102960004546E0B5CA4B8FB003931B78FF2B00D1CF
:1029700046E1C84BC84E9B465F46C84B0BAC029322
:10298000C74B019335686A69EFF3108172B613681B
:10299000002BFCD0BFF35F8FA9612800210000F05D
:1029A000C3FF6A69AB69BFF35F8F0021116083F3D6
:1029B0001088002800D123E16378082BE2D89B001F
:1029C000FB589F466368002BDCD0A0689847D9E786
:1029D0007F222179B14D0A405300EB189846C8096F
:1029E000804440460123303005799D4305710579C7
:1029F00003339D430571002A00D108E14346A94AEB
:102A00001B7D1278934200D3F8E0A74A5B0115685A
:102A1000ED18002D00D1F3E0A36862792078AD694C
:102A2000A847AFE7A14A1378002B00D1E8E013785C
:102A3000013BDBB213701378002BA3D10122974D19
:102A400001212B78042013432B703423EA5C8A4342
:102A5000EA54EA5C8243EA540133EA5C8A43EA546A
:102A6000EA5C8243EA5423780020984600F05EFC3A
:102A7000602223791A40602A00D1F3E0402A00D175
:102A8000F9E0DB06DB0E012B00D117E1022B00D1B0
:102A9000CCE0002B00D0E5E0202A00D10FE2002A94
:102AA00000D0DFE06379092B00D9DBE0804A9B008E
:102AB000D3589F46794D2B78DB0700D462E7FFF7A8
:102AC000C3FE5FE7029BDB78DB0700D45AE7606850
:102AD000FFF7ACFE56E7714D2B78DB0700D451E7CA
:102AE00028780007C00FFFF7ADFE4BE723786C4A4C
:102AF000984693466B4B6C4A9946310092463A0091
:102B000046464F460025914688461B780EE05346C0
:102B10001B686A019B18002B00D17EE0DB68300047
:102B2000984701353B78EDB2AB420CD39D42EED3D2
:102B3000EB1A5B015B44DB683000984701353B785A
:102B4000EDB2AB42F2D2554D542200212800FFF7DE
:102B50000BFB1022FF21281DFFF706FB2800202277
:102B6000FF21143046464F46FFF7FEFA00F0D4FB33
:102B70002379AB7006E723784B4A9846494B924637
:102B800099463200BB46464600254F4690461B7884
:102B90000DE053461B686A019B18002B41D0DB688F
:102BA0003000984701353B78EDB2AB420ED3AB42D3
:102BB000EFD8019AEB1A94465B016344DB6830005E
:102BC000984701353B78EDB2AB42F0D2029D5422DA
:102BD00000212800FFF7C8FA1022FF213548FFF72F
:102BE000C3FA28002022FF21143046465F46FFF733
:102BF000BBFA00F091FBFFF723FEC3E6934213D02C
:102C00000FB0F0BCBB46B246A946A046F0BDA368D3
:102C10006279207800F09EFBB4E646464F461F4D91
:102C2000A4E746465F46E4E71D4DF5E67023217AAA
:102C30000B4217D1C80983460F330B405B009946FE
:102C40001848EB185B441B7D0078834261D216481C
:102C50005B01006882469A44002A00D14EE1534647
:102C6000002B5ED120780021FFF766FD80212078BF
:102C7000FFF762FD86E6104800F058FB0121404650
:102C80000CAAFFF7CFFD002800D07BE6EAE7C0469C
:102C90009C1000207C4D0010741E00201C1E002083
:102CA000244E0010A0240020AC1C0020A2240020F0
:102CB000A04D0010201E002025280010237A0F2B85
:102CC000D0D8D54AEB181B791278934234D3C9D1A6
:102CD000D24D686900F02AFB012140466B690CAABD
:102CE0009847002800D04DE66022150023791D404A
:102CF0001A42B7D163790A3B012BB3D800F016FB17
:102D000063790A2B00D17DE140460CA900F09AFAC4
:102D100038E6834200D0ECE0C04B9A46002A00D14E
:102D2000ECE05346586900F001FB53460121404650
:102D30005B690CAA9847A6E7B94A5B011568ED18CC
:102D4000002DC6D18EE7A3799A466B789A45DBD0E1
:102D50006B78002B00D028E153466B70002B00D11C
:102D600020E150460138C0B2FDF70AFE002800D12C
:102D700071E14378022B00D06DE10122C179A946AF
:102D80008B11491113400A40302112015B0113439A
:102D90002A788A4313432B7009239B4683445D465C
:102DA000B346C37882781B021343C31806939A4B29
:102DB00004970593994B0893994B9A46994B09931D
:102DC000069BAB4200D849E16B7801220B2B03D163
:102DD0002B78EA78ED186B78042B00D038E1069B4D
:102DE00000265B1B9BB20793059B17001B7818E01E
:102DF00053461B6872019B18002B00D128E1290063
:102E000040461B69079A9847082803D9079B8342C5
:102E100000D30BE1059B01361B78F6B2B34200D21A
:102E200016E1B342E4D8089AF31A94465B0163446E
:102E3000E5E76B780AAA02321370404601230CA919
:102E400000F016FA9EE5E3881A0AD8B20F2A00D9D4
:102E500008E775499300CB589F460CA800F06CFA20
:102E60004046A179FFF7A2FB02222B7813432B7077
:102E700088E5E388012B00D0F4E608222B78404651
:102E800093430CA92B7000F0DDF97BE50220297833
:102E90000AAB9A1C8B068908DB0F01400B43138099
:102EA000404602230CA900F0E3F96BE5E388012B0F
:102EB00000D0D7E608222B7813432B7024E7237A1F
:102EC0000F2B00D9CEE6544AEB181B7912789342A7
:102ED00028D2534A5B011568ED18002D00D1C1E6D8
:102EE000686900F023FA012140466B690CAA9847F3
:102EF000C9E6002A00D0B5E600239A46627902208E
:102F0000130004928343012B11D0002A00D0A9E6BC
:102F10002B004B445B4430331B790AAA9B07DB0F21
:102F20000232BCE7934200D09CE63C4DD8E7E388F0
:102F3000002B12D1039B1878049B012B23D0FFF7A1
:102F4000FBFB4B460221EB185B4430331A790A43F2
:102F500001211A711A790A431A715346002B00D1C4
:102F600010E5586900F0E2F9534601215B690CAAAB
:102F700040469847002000F0D9F93523EB5CDB0789
:102F800000D5FFE4C0E6FFF7F5FB4B460221EB1846
:102F90005B4430331A798A431A711A7904998A4347
:102FA0001A71DAE7FFF74CFCAEE600214046FFF766
:102FB00007FB4046FFF7AAFB00229346174AAB786F
:102FC0000592174A049306922A00134B5D469946D0
:102FD00093461B780EE0069B6A011B689B18002B2A
:102FE00055D0DB68404698474B4601351B78EDB21B
:102FF000AB4238D39D42EED3059AEB1A94465B015F
:103000006344EEE70AAB9A1C404601230CA91570F5
:1030100000F02EF9B6E4C046A0240020244E001093
:10302000AC1C0020301E0020C84D00103A000700E4
:10303000002A3CD0AB789A18D2B204E00133DBB25C
:103040000E719A4233D04946C9180879FF28F5D045
:103050005E464D46049F00236B7003E65E46049F68
:10306000FFF7ECFB50E65D46542200212800FFF7F5
:103070007BF81022FF21281DFFF776F82800202278
:10308000FF211430FFF770F8049BAB7064E65D46D7
:10309000FAE7FFF7CDFB021E00D1E3E5D378917884
:1030A0001B020B4340460CA900F0E2F8EBE53300AD
:1030B00029003A00099800F01DFC059BED191B78CA
:1030C000B34200D37CE6C3E7FFF7B4FB021E00D196
:1030D000C8E5404613780CA900F0CAF8D3E5218969
:1030E000FDF756FC021EF4D1BCE5022A0FD0FFF713
:1030F000A3FB021ED2D1B5E5FDF746FC021E00D1AE
:10310000B0E5122340460CA900F0B2F8BBE5FDF78C
:1031100037FC021EC2D1A5E5F8B557464E46DE463D
:1031200045460C00E0B516001F00002A3CD0702375
:1031300098461E4B00259B461D4B9A461AE05B465F
:103140001B78200099465346997800F095FB00289B
:103150001CD021004846FFF74FFA002816D0A3786C
:10316000DA09012A19D00A9A013513702378E41874
:10317000B54219DA6378052B08D1E3789B079B0FDA
:10318000BB4203D14246A3781A42D8D00020F0BCFB
:10319000BB46B246A946A046F8BD0B9A013513704E
:1031A0002378E418B542E5DB0120F0E79C1000200D
:1031B0001C1E00200B007F2010B51840DB093433A3
:1031C0004000044AC018044B1168C01800F02CFBE2
:1031D00010BDC046701E00201C1E002070B57F244C
:1031E0000F480C4064000419CD096419303420796B
:1031F000C00701D5002070BD012625790948354357
:1032000000782571FFF786FA0028F4D1012223798E
:10321000934323712379033293432371EAE7C04632
:103220001C1E00209C1000207F22054B0A405200EB
:10323000C9099B185B1830331879C007C00F704755
:103240001C1E002070B5094C0600082220000D004D
:10325000FEF790FF00238021E360A3602B7830000D
:10326000994300220023FFF7B9FF70BDF01C002036
:10327000F8B5CE4647469046254E80B58146082291
:1032800030000D001F00FEF775FF4346B3600023BA
:10329000F381EC79AB7924021C43231CBC4200D996
:1032A0003B1C9FB2B381002C0DD0002F17D042469B
:1032B000002A2BD0402F1BD89FB233787F2B1CD8ED
:1032C0000021144A0FE080212B78002299434846C0
:1032D0000023FFF783FFC0BCB946B046F8BD7F238B
:1032E0000022317899433B004846FFF777FFF2E729
:1032F00040239FB233787F2BE2D9064C3A004146F7
:103300002000FEF737FF80212200ECE70020E2E7F3
:10331000F01C0020B01C002010B51422002102482F
:10332000FEF722FF10BDC046F01C0020014B1861C3
:103330007047C046F01C002010B5054C0100082263
:103340002000FEF717FF0023A360E36010BDC04616
:10335000F01C002070B5384C1D0023780600DA09F7
:10336000C9098A4210D00020002D00D070BD210074
:103370003000FFF733F92369002B03D0220003212B
:10338000300098470120F1E77F2B06D8A06800287D
:1033900034D02A002949FEF7EDFEE289A1685219CE
:1033A000E38892B24919E281A160934214D03F2D83
:1033B00012D9A389981A051C80B240282AD82078EF
:1033C000ADB27F2828D800219A4232D01B4A2B0068
:1033D0003000FFF703FFC9E72369002B05D0220067
:1033E00002213000984700280AD08021237800224B
:1033F000994330000023FFF7F1FEB7E70020B5E75F
:1034000000213000FFF798F930008021FFF794F990
:103410000120ABE74025D2E79A4207D0074C2A00AB
:103420002000FEF7A7FE80212200D0E780210022A5
:10343000CDE70022CBE7C046F01C0020B01C0020E6
:103440007047C046012070477047C0467047C0466D
:1034500042000C4B1218920010B59B185C78FFF7D5
:10346000F5F9002801D1002010BDFFF7F7F9002879
:10347000F9D1002CF7D02100FFF7D6FE01235840E8
:10348000C0B2F1E7041E0020F0B50E0004001500E4
:10349000190083B0002B2BD06B460622981CFEF738
:1034A00069FE002C02D0002003B0F0BD154F0020B3
:1034B0007978FFF77FFE0028F5D0002E0CD16B46FF
:1034C000114A1D705E7003CB03C208230E4A79783F
:1034D0000020FFF783FEE7E7402369460B480822F8
:1034E000C65441300D704C70FEF744FE0923EDE7E1
:1034F0006B461A70597006220021981CFEF734FEA4
:10350000CFE7C046041E0020841D0020441D00207B
:1035100010B50C2200210248FEF726FE10BDC04661
:10352000041E00200120704710B50C220021024823
:10353000FEF71AFE10BDC046041E0020F0B54B7900
:1035400006000D0083B0032B0AD10879C400241AA9
:103550001234A4B2944203D8194F7B78002B03D0C5
:103560000024200003B0F0BD097869184B78212BA6
:10357000F6D1B9600B780200C9187B1C0193BB1C03
:10358000009330000323FFF7C7FD0028E8D0AB7994
:10359000012B01D1EB79FB700123BB71AB78B978BA
:1035A0003B70BB68DA791B7A1B021343BB8000298E
:1035B000D7D040233000034AFFF710FED1E7C046C2
:1035C000041E0020C41D00201F23F0B51400127833
:1035D000050083B01340012B01D000200CE05A4EAF
:1035E000207933789842F8D16023180010401342B4
:1035F00004D101290BD0012003B0F0BD2028ECD16B
:1036000063780B2BE9D8514A9B00D3589F466378C7
:10361000062BE2D1E378212B7AD0222BDDD10020BA
:10362000FDF7AAF921000200B3882800FFF720FE69
:10363000E1E7012910D00329DDD1A1780020B17183
:10364000FFF7FEFED7E70129D5D1E1780020F1711F
:10365000FFF7F8FE0028C0D021002800FFF7F2FD98
:10366000C9E701295ED00329C5D1E079A379000219
:103670001843E278A178041C402800D94024344B38
:10368000A4B2002907D0012805D91878884202D1B0
:10369000013C304BA4B200200094FDF76BF9AAE77F
:1036A0000129A8D10123210028002B4AFFF7E0FDC2
:1036B000A1E701299FD1012321002800274AFFF714
:1036C000D7FD98E7012996D1E379A0791B0203433E
:1036D000E278A178181C402B00D9402080B2002944
:1036E0002DD0012B2BD90126194F0138397080B20A
:1036F0007B1C00900020FDF73BF933189BB2002B98
:1037000000D16AE73A0021002800FFF7B1FD72E717
:10371000B268002A00D160E7210028001378FFF783
:10372000A7FD69E7E379A2791B021343402B00D977
:1037300053E721002800064AFFF79AFD5BE7044F94
:1037400000263B00D5E7C046041E0020444E001072
:10375000441D0020451D00200A1E00200B1E0020D5
:1037600070B51B4D0400A8786E7882B0884204D0F2
:103770008E4216D0002002B070BD9BB2864211D09E
:10378000144E002A17D1009300213300002002328A
:10379000FDF7F0F8402332002000A978FFF71EFD66
:1037A000E9E79BB2002A0CD100201A000A49FFF772
:1037B0004BFE0120DFE7320002210020FFF746FE2A
:1037C000E8E700200121044AFFF740FE0120D2E78C
:1037D000041E0020C41D0020841D002000B503002D
:1037E00083B0002910D00020012B07D80A78002AC6
:1037F00004D00C48C2540120012A01D003B000BDFE
:103800001800FFF733F8F9E701236A46002001A901
:103810009380FFF72BF80028F0D00122014B1A709B
:10382000ECE7C046101E0020037870B5DB070400EB
:103830000E00DD0F002B17D103785B0701D52800A0
:1038400070BD01213000494200F052FF2378DB07B0
:10385000DD0F002B0AD123785B0708D404222378DC
:1038600001251343237002E00025E8E7002530001E
:1038700000F01EFFE3E7C046437902791B021343C1
:10388000C2785B0592075B0D920F022A1DD0032AB6
:103890000CD00020012A08D102394A425141124A73
:1038A0009446614499424041C0B2704702394A1E71
:1038B00091410E4A494211408022D2009446002094
:1038C000614499424041C0B2EFE7022905D000208F
:1038D00040229A424041C0B2E7E7054A9818434265
:1038E0005841C0B2E1E7C046FF03000040FCFFFFC3
:1038F00000FEFFFF8A1870B5914207D27F264C78F0
:10390000052C04D00C7809198A42F8D870BD34000F
:103910008D782C4064000419ED0963550C78091961
:103920008A42ECD8F2E7C04670B5040000690E0088
:10393000002803D00121494200F0DAFE2589608980
:10394000A288A9B283B2854232D3CD1AADB2002D7E
:1039500028D0AA4208D291422FD3891A8BB2638110
:103960009A4203D89B1A9BB29A42FBD9E2882168FB
:103970005204520C53433000C918FEF7FBFB638915
:103980000125591C89B2A2888B420DD90021520011
:10399000891A89B220696181002801D000F088FE6F
:1039A000280070BD618989B252009142F2DBEFE7D5
:1039B0005500ED1A4D19ADB2C9E789188BB2638174
:1039C000CEE7C046F8B50400C0680E00002803D05A
:1039D0000121494200F08CFE258920896189A28855
:1039E000ADB283B28FB2884229D3DB1B9BB29A421D
:1039F00009D8E779FF0906D1E068002801D000F076
:103A000057FE3800F8BD2B0095421DD39B1A9BB280
:103A10009342FBD2E28820685204520C5343310097
:103A2000C018FEF7A7FB6B1C9BB2A2889D4217D95A
:103A3000002352009B1A9BB201272381DCE751002F
:103A4000C91B5B189BB2D2E7E28820685204520C73
:103A500053433100C018FEF78DFB0135A288ABB28D
:103A600052009342E8DBE5E710B50400C068002887
:103A700003D00121494200F03BFE2069002803D019
:103A80000121494200F034FE0023E0686381238174
:103A9000002801D000F00CFE2069002801D000F0C1
:103AA00007FE012010BDC04610B583070AD00300F1
:103AB000032102E001330B4205D01A78002AF9D124
:103AC000181A10BD030019680C4A0D4C8A188A4355
:103AD00022420FD15968094A04338A188A43224284
:103AE00008D15968054A04338A188A432242F1D022
:103AF00000E001331A78002AFBD1E1E7FFFEFEFE69
:103B000080808080034B10B51A680123503200F08A
:103B1000B3FC10BDA010002010B5034B01001868C5
:103B200000F07AF810BDC046A01000200323CAB2EE
:103B3000F0B50340002A35D00324002B2DD1FF23FC
:103B40000B401D02ED182B04ED182C000168264EC9
:103B50004C408B198B43A119A143244E0B43334294
:103B600011D14168204F0C00CB196C408B43E119F7
:103B7000A1430B4304303342F3D00378002B05D02C
:103B80009A4204D001300378002BF9D10020F0BD17
:103B90009342FCD001302042D1D00378002BF7D1E2
:103BA0000020F4E7002B08D0032202E0013010428D
:103BB00003D00378002BF9D1E9E702680A4B0B49DF
:103BC000D31893430B4206D14268074B0430D318F5
:103BD00093430B42F8D00378002BD8D043780130C0
:103BE000002BFBD1D3E7C046FFFEFEFE8080808025
:103BF00070B5074C074D641BA41005D0013CA30011
:103C0000EB589847002CF9D100F040FD70BDC0463C
:103C1000984700109847001070B5040008000D0088
:103C2000FFF742FF461C3100200000F009F8041E97
:103C300003D032002900FEF79DFA200070BDC04677
:103C4000F0B54E464546DE465746E0B50D000B350D
:103C5000060085B0162D27D8102900D9DAE000F02B
:103C60005DFC102518230221C74FFB181A005C6861
:103C7000083A944200D146E103226368A168934365
:103C8000E268CA6091600121E3185A6830000A4373
:103C90005A6000F045FC2000083005B0F0BCBB467F
:103CA000B246A946A046F0BD07239D4300D5B1E02A
:103CB000A94200D9AEE000F031FCFC235B009D423C
:103CC00000D294E1690A00D1A8E0042900D94FE1AB
:103CD00038239846A90988443931CB00082252423A
:103CE0009446A94FFB189C446346DC68A44514D055
:103CF000032399460B0061469C4607E0E068002AD2
:103D000000DBFAE0814200D1FBE004004A46636830
:103D100093435A1B0F2AF1DD41463A003C690832B1
:103D2000944200D1D8E0032063688343581B0F28D6
:103D300000DD60E13A617A610028A4DA7A68904691
:103D400080229200934200D3E3E0DA08580901236D
:103D50008340404618438046D300DB199A68786058
:103D6000E360A2609C60D46001208B1098404045C5
:103D70005CD8434603420AD103239943434640009B
:103D80000431034203D1400004310342FBD003233A
:103D9000B3469C460E00B8460190F0004044010036
:103DA000B246CB680BE064465A681F00A243DB684A
:103DB000541B0F2C00DDEDE0002C00DB07E19942E5
:103DC000F1D101239946CA44534608319B07E8D1F3
:103DD000032205E003680838013E834200D001E277
:103DE0003242F7D14346019A5B689343424653609F
:103DF000019A520001929A4216D8002A06D113E085
:103E000004229146019ACA44520001921342F7D00B
:103E10005646C2E70C23002033603EE780233F2252
:103E2000402190469B0059E75E4647460322BC6806
:103E3000636893439846AB4202D35A1B0F2A4EDC69
:103E4000230043440293514B08209A461B681033C9
:103E50005B19019300F0C4FB4D4903900B688B463E
:103E6000013306D08446019B4242013B6344134028
:103E700001933000019900F055FB030081460133A6
:103E800000D1D6E0029B834200D9D0E053465A6865
:103E9000019B51469C4662444A600298039901394D
:103EA000484500D0E3E04846084200D0DFE0B9686A
:103EB0004344894601210B4349464B605146C96A38
:103EC000914201D25146CA625146096B914201D2D8
:103ED00051460A634C46AEE07B68984644E70123AE
:103EE00029001A431943651961603000BD606A609A
:103EF00000F016FB20000830CFE6A268D060826098
:103F0000C1E6614609E7DC680231A34200D104E75B
:103F1000B2E65A0A042A00D882E0142A00D907E13E
:103F200010005B3082465C32D2000820404284465A
:103F3000BA189444624692680B308146944500D189
:103F4000DEE00800A2466146844602E092689142A3
:103F500004D04C465068A0439842F7D8D3686146D5
:103F600054469C466346A260E3609C60D460FBE6D6
:103F700014296DD9542900D9E3E06E239846290B02
:103F800088446F31CB00A9E6F0110020E01A002030
:103F9000E8110020BA4601205146844649190543DC
:103FA00050464560856847466046EB605E469D60CA
:103FB000534639617961204308374860CF6030004B
:103FC0008F609C5000F0ACFA5046083065E6BA4667
:103FD00001205E465244516801435160BA68300086
:103FE000D3609A6000F09CFA3800083055E62B0048
:103FF000E908083338E66119884601218C460D43EB
:104000004146656039617961CA608A6062460243EF
:104010004A60E050300000F083FA200008303CE6AF
:104020009A091000393238308246D2007DE7BC420E
:1040300014D0BC686368032293435A1BAB4202D37B
:104040000F2A00DD4BE7300000F06AFA002024E67A
:104050005B23984688445C31CB003FE653465A6860
:10406000019B9C46534662445A60039B591E5B4623
:104070001B68013370D04B4602981B1A9B1852469E
:10408000536007234A4648461A400292184240D0DD
:104090000398013384469B1A019A99444A44019239
:1040A00063440A409B1A194030008B4600F03AFAEC
:1040B000431C77D04B46C01A03005B440193534620
:1040C0005A6801205A445A604B464946BB60019BDE
:1040D00003434B60BC4200D1F0E643460F2B3FD96F
:1040E00007210C3B8B436168014005201943616047
:1040F000E118486088600F2B49D84B465B68DDE6C5
:104100005346981001238340404618438046786008
:1041100028E7019B039A4B440B40D31A1940300007
:104120008B4600F0FFF9431CC4D100239B46C6E731
:10413000542A17D81A0B10006F326E308246D20004
:10414000F3E6AA235B00994217D8DD3B9846E90BBA
:1041500088447831CB00C1E55B464A461A6090E757
:10416000486070E7AA204000824226D8DA0B10008F
:10417000783277308246D200D7E61C4B994226D857
:104180007C239846A90C88447D31CB00A6E521000C
:104190003000083100F086F853465A68BB689946EB
:1041A0005B688BE6019A029B94464A46083B63444F
:1041B0009B1A019300239B4681E70C4882420CD84E
:1041C0009A0C10007D327C308246D200ADE6FE2390
:1041D0007E227F2190469B0080E5FE227E20920079
:1041E0008246A2E643465B6802E6C04654050000EC
:1041F000F0B5C646060000B508200D0000F0F0F945
:104200000400300000F08AF9234B210098469B6897
:104210005F6803239F4338001138401B0019FDF7E6
:1042200089FC451E6543AC4208DC0021300000F0EB
:1042300079F943469B68DB19984206D0300000F0BC
:104240006FF9002080BCB846F0BD3000694200F034
:1042500069F901300ED0012243467F1B9B6817434A
:104260000E4A5F60136830005B1B136000F058F962
:104270000120E7E70021300000F054F943469A6836
:10428000831A0F2BDADD064C04492468001B0860F2
:1042900001210B435360D1E7F0110020E41A002004
:1042A000E8110020F8B5CE46474605000C0080B561
:1042B000002957D000F032F9012321009C4608392B
:1042C00048686246030003249343CF187A68654E1A
:1042D000A243B468BC4200D170E0BC18A146644659
:1042E0007A60044221D10868091A1B188868804640
:1042F000484640682040340008348146A04551D0EB
:104300004046CC68C460A0604846002811D19B1884
:104310005548BA68824200D17FE0F868D060826078
:1043200001221A434A60CB5007E0484640682042C9
:10433000EDD062461A434A603B608022920093426D
:1043400014D2DA085809012383407068034373606C
:10435000D3009B199A68CB608A609960D16028006D
:1043600000F0DEF8C0BCB946B046F8BD5C0A042CCB
:104370003DD89C09200039343830E40034192268D3
:10438000083C0327944203D140E09268944203D052
:104390005068B8439842F8D8D468CC608A60A1606D
:1043A000D160DCE7002858D1B868D218FB68C36038
:1043B0009860634613434B608A50D0E79A1863466F
:1043C000034206D10B68C91A8868D218CB68C3604B
:1043D0009860012313434B60244BB1601B689342E8
:1043E000BDD8234B28001968FFF702FFB7E7142C4C
:1043F00007D9542C1AD81C0B20006F346E30E400FF
:10440000BCE720005C345B30E400B7E70123801098
:104410008340706803437360BFE7D1609160CA60F6
:104420008A6001221A434A60CB5098E7AA225200C0
:10443000944205D8DC0B200078347730E4009DE707
:104440000C4A944205D89C0C20007D347C30E4005A
:1044500094E7FE247E20A40090E762461A434A6057
:104460003B607CE7F0110020F8110020EC110020E7
:10447000E01A002054050000F0B5002826D00700FF
:1044800038000C000678013702E00134AE4214D047
:104490002578002DF9D1002E1DD03E000B00357877
:1044A000013702E00133002CF7D01C78A542F9D186
:1044B0000023002D06D11360F0BD002BE0D1176062
:1044C0000370F9E700213B003170F4E71068002821
:1044D000D5D10020F0E700201660EDE710B50123EC
:1044E000FFF7CAFF10BDC046014B18687047C046B1
:1044F000A010002010B5034B01001868FFF7A0FBC7
:1045000010BDC046A010002010B5034B0100186874
:10451000FFF7C8FE10BDC046A01000207047C0467F
:104520007047C046002370B5064C050008002360A4
:10453000FDF748FE431C00D070BD2368002BFBD064
:104540002B60F9E7141B002010B5010000230022A6
:10455000002000F053F810BD024670B50A439207E0
:104560002AD11E4DEE0104C808C9541B944334409F
:1045700017D0D0B2D9B2401A2106014310D190B25F
:1045800099B2401A210401430AD110021902000A0B
:10459000090A401A2102014302D1100E190E401AD5
:1045A00070BD9A42DFD010BA19BA884201D90120F1
:1045B00070BD0020C04370BD02780B78013001311E
:1045C000002A09D09A4207D102780B7801300131D4
:1045D000002A01D09A42EFD0D01A70BD010101012A
:1045E000802310B55B01082801D1180010BDFFF72A
:1045F0007BFF16230360173BF7E7C046F0B5C646BE
:104600001A4C00B52568002D2AD06C681F2C2ADCB6
:10461000002808D10020631C0234A4006B606151A3
:1046200080BCB846F0BD8827A600AE19F25101370C
:10463000FF37BC460122AC446746A2403F68904623
:1046400017436246176084277F00F3510228E1D1A7
:10465000280042468D30FF30036813430360D9E7DA
:10466000034D2560D1E701204042D9E7A81C002076
:10467000181B0020034B10B5002B02D00248FFF797
:1046800063FF10BD00000000F13B0010F8B5C0460C
:1046900001B40248844601BC604700BF0503002006
:1046A00001B40248844601BC604700BF450C0020AD
:1046B00001B40248844601BC604700BF29020020C3
:1046C00001B40248844601BC604700BF5D0F002072
:1046D00001B40248844601BC604700BF4104002089
:1046E00001B40248844601BC604700BF5D0F002052
:1046F00001B40248844601BC604700BF9D01002010
:1047000001B40248844601BC604700BF0501002097
:1047100001B40248844601BC604700BFD50C0020AC
:1047200001B40248844601BC604700BF1D0C002054
:1047300001B40248844601BC604700BF850C0020DC
:1047400001B40248844601BC604700BFC10000209C
:104750001519001041190010251B001059210010D7
:10476000A51F0010A92000104D1A00105D1900109F
:104770007D19001091190010B90E00109919001040
:1047800071120010DD180010650B00107546001046
:08479000C5240010FD02001019
:1047980021402324255E262A28295F2B7B7D7C3A0D
:1047A800223C3E3F7E0000002B0000006374726CC8
:1047B80000000000636F6E74726F6C00616C7400AF
:1047C80073686966740000006775690077696E0030
:1047D800636D640064656C0064656C6574650000F5
:1047E800656E74657200000071756F746500000075
:1047F8006374726C2B616C742B7400006364207E8C
:104808000A0000006563686F202223212F62696E09
:104818002F736822203E2064656D6F2E73680A002E
:10482800636C6561720A00006563686F20226563C6
:10483800686F20796F752068617665206265656E9E
:10484800206861636B65642122203E3E2064656DAB
:104858006F2E73680A0000006563686F2022656325
:10486800686F206769766520323020555344206987
:104878006E20626974636F696E20746F2074686556
:1048880020616464726573733A22203E3E20646539
:104898006D6F2E73680A00006563686F2022656378
:1048A800686F2062633171656D6D3733396C6335BC
:1048B800763630767539653873347037377A6C7276
:1048C8006172727135667968633377723022203E7F
:1048D8003E2064656D6F2E73680A00006563686F1B
:1048E80020226563686F206265666F7265206920A3
:1048F8006F626C697465726174652065766572793A
:104908007468696E67206F6E20796F757220636FA7
:104918006D70757465722122203E3E2064656D6F4E
:104928002E73680A000000006563686F20226563C3
:10493800686F206861726D6C6573732064656D6F54
:104948006E7374726174696F6E206F662074686527
:10495800207069636F207275626265722064756386
:104968006B7922203E3E2064656D6F2E73680A00C5
:1049780063686D6F64202B782064656D6F2E736893
:104988003B20636C6561723B202E2F64656D6F2E32
:1049980073680A0052617370626572727920506997
:1049A800000000005069636F204B6579626F617287
:1049B8006400000031323334353600000A2A2A2ACE
:1049C8002050414E4943202A2A2A0A000A000000A2
:1049D8004E6F207370696E6C6F636B7320617265C4
:1049E80020617661696C61626C650000486172647F
:1049F8007761726520616C61726D20256420616C3D
:104A0800726561647920636C61696D65640000009A
:104A180048617264206173736572740052656C65D5
:104A280061736500626F6F74325F77323571303849
:104A380030000000322E322E300000007069636FA3
:104A4800000000007069636F5F7275626265725F73
:104A58006475636B790000004A756E203139203225
:104A680030323600556E68616E646C656420495258
:104A78005120307825780A0065702025303258207A
:104A880077617320616C7265616479206176616910
:104A98006C61626C6500000043616E277420636F6F
:104AA8006E74696E75652078666572206F6E206910
:104AB8006E61637469766520657020253032580010
:104AC8004C4544009C03001084030010320300107E
:104AD80032030010320300103203001032030010BA
:104AE80032030010320300103203001032030010AA
:104AF800320300103203001032030010320300109A
:104B08003203001032030010320300103203001089
:104B18003203001032030010320300103203001079
:104B2800A4030010900300106803001098030010FD
:104B380094030010880300107C0300106803001021
:104B48007803001074030010800300105003001055
:104B5800700300106C030010580300105403001079
:104B680074030010420300104203001042030010B7
:104B780042030010420300104203001042030010D9
:104B880042030010420300104C0300104C030010B5
:104B98007003001050030010580300105403001055
:104BA800A00300103C0300103C0300103C0300105D
:104BB8003C0300103C0300103C0300103C030010B1
:104BC8003C0300103C0300103C0300103C030010A1
:104BD8003C0300103C0300103C0300103C03001091
:104BE8003C0300103C0300103C0300103C03001081
:104BF8003C0300103C0300103C0300103C03001071
:104C08003C0300103C0300103C030010600300103C
:104C180048030010640300108C0300106C0300109C
:104C28005C03001036030010360300103603001032
:104C38003603001036030010360300103603001048
:104C48003603001036030010360300103603001038
:104C58003603001036030010360300103603001028
:104C68003603001036030010360300103603001018
:104C78003603001036030010360300103603001008
:104C880036030010360300103603001060030010CE
:104C980048030010640300105C03001012010002B6
:104CA800000000408A2E0A000001010203010000F2
:104CB80009022200010100A03209040000010301D9
:104CC8000100092111010001224300070581034069
:104CD800000A000005010906A1018501050719E080
:104CE80029E71500250195087501810295017508C8
:104CF800810105081901290595057501910295019C
:104D080075039101050719002AFF00150026FF0009
:104D1800950675088100C00009040000060052507D
:104D2800D3F07542244A001006005250E182887F71
:104D38002C4A001006005250ABB360533C4A001096
:104D480006005250BBFF3CB6444A001006005250C1
:104D5800861C03024C4A0010060052505422A29DA1
:104D6800604A001005005250DE65F468EC640010DB
:104D78000D0A000084290010EC2A0010762B001080
:104D8800C42A0010D62A0010B42A0010242A0010C1
:104D9800D0290010C42900108C2E0010722E00108B
:104DA800642C0010AC2E0010642C00105A2E001039
:104DB800462E0010642C0010322E0010462D0010D4
:104DC800642C0010F8300010EA300010DE300010BB
:104DD800642C0010642C0010C8300010EA30001059
:104DE800642C0010642C0010642C0010642C00103B
:104DF800642C0010642C0010642C001092300010F9
:104E0800A20D0020A20D0020EC0D00200C0E0020A9
:104E18004A0E00205C0E0020980D002000000000C3
:104E28001135001025350010293500103D350010CA
:104E3800C93500106137001000000000DA35001095
:104E4800C4360010B2360010A0360010DA35001053
:104E5800DA350010DA350010DA350010DA350010CE
:104E680062360010463600103236001009005250E3
:104E780000000002C84A0010002020202020202026
:104E880020202828282828202020202020202020F2
:104E98002020202020202020208810101010101002
:104EA800101010101010101010040404040404044E
:104EB80004040410101010101010414141414141E8
:104EC80001010101010101010101010101010101CA
:104ED80001010101101010101010424242424242DA
:104EE800020202020202020202020202020202029A
:104EF8000202020210101010200000000000000042
:104F08000000000000000000000000000000000099
:104F18000000000000000000000000000000000089
:104F28000000000000000000000000000000000079
:104F38000000000000000000000000000000000069
:104F48000000000000000000000000000000000059
:104F58000000000000000000000000000000000049
:104F68000000000000000000000000000000000039
:0C4F78000000000000000000000000002D
:104F8400244D0010304D00103C4D0010484D0010D1
:104F9400544D0010604D00106C4D0010744E001004
:104FA400D02330B500251B0600245D5705E0BFF370
:104FB4005F8F1C6081F3108820BF0268EFF31081BB
:104FC40072B61368002BFCD0BFF35F8F02790368BD
:104FD4007F2AECD90571BFF35F8F00221A6081F339
:104FE400108830BDF0B5C646150000B504001E009B
:104FF4000268EFF3108172B61368002BFCD0BFF384
:105004005F8F0423E3562268002B2BDBBFF35F8FF3
:105014000020106081F31088D02212061278002735
:1050240052B290469A420ED1002080BCB846F0BDE0
:10503400BFF35F8F176081F310882800310000F000
:10504400FFFE0028F0D12268EFF3108172B61368D6
:10505400002BFCD0BFF35F8F237922687F2BE7D925
:10506400434602E0D0231B061B682371BFF35F8F06
:105074000023136081F310880120D6E7F0B5C646FB
:1050840000B50D00040000F0EBFEFA2206000F004C
:10509400002328000021920000F0F2FE36184F4150
:1050A400002F02DA0126174F7642D0231B061B6815
:1050B400002598460AE0BFF35F8F156081F31088DE
:1050C4003000390000F0BCFE002818D12268EFF34C
:1050D400108172B61368002BFCD0BFF35F8F237965
:1050E40022687F2BE7D943462371BFF35F8F0023E8
:1050F400136081F31088012080BCB846F0BD002005
:10510400FAE7C046FFFFFF7F0268EFF3108172B633
:105114001368002BFCD0BFF35F8FFF230371036878
:10512400BFF35F8F00221A6081F3108840BF70477D
:1051340010B5084C2378002B0AD180230648074970
:105144005B051A68C25004338B42FAD101232370E1
:1051540010BDC046A3240020381F00100001001019
:1051640010B5014B984710BD391F0020064B5A68F3
:1051740002609A684260DA6882601A69C2605A6999
:1051840002619B6943617047000002400268064B5C
:105194005A6042689A608268DA60C2681A61026979
:1051A4005A6142699A61704700000240034B1A68D1
:1051B400C0239B009343024A136070470C80014054
:1051C4000C900140054B1A6880239B005340C02279
:1051D40092001340024A13607047C0460C8001409D
:1051E4000C9001400023F0B5DE4657464E46454636
:1051F4009A46E0B589B001900E00988A45491B8B08
:1052040014009847534681464349988A1B8B984714
:10521400534642490500988A1B8B98478046FFF7FE
:1052240087FF02A8FFF7A2FFC847A847FFF7CAFFF6
:10523400251E22D00823C0219C460220490562462F
:105244008B6A1A4018423FD0631B002D2FD1002ACD
:1052540011D1002C11D0C0235B059B4602239A4632
:10526400063399465B464A4657469B6A1A401F4294
:1052740042D0002AF6D0002C30D1FFF797FFC04768
:10528400FFF76EFF02A8FFF781FF09B0F0BCBB4631
:10529400B246A946A046F0BD002C2FD1C02252052B
:1052A400926A914608224F463A40BF072DD50D2BEE
:1052B4001BD9002AF0D1C0225205926A91460822D5
:1052C4004F463A40BF07F2D4002A04D12B002343AF
:1052D400002BB4D1D1E72B00002CF9D00B6E013C8C
:1052E4003370230001362B43F2E7019F013D3B78E5
:1052F40001370B660197E7E70025E5E7C0235B0567
:105304001B6E013C3370013699E72B00002ADFD174
:10531400DCE7C0464946000045580000464300000B
:105324000022154B10B59A60DA601A615A619A61CD
:10533400DA611A625A629A62DA621A635A639A6387
:10534400DA631A645A649A64DA641A655A659A6567
:10535400DA651A665A669A66DA661A675A679A6747
:10536400DA67F03292000021044800F0A1FD044BFA
:10537400044A1A6010BDC04600001050B820002036
:105384007C24002080011050F0B54E464546DE4690
:105394005746E0B5214B00249E6D012585B0002EB3
:1053A40022D01F4B9A46012399461E4B984601E092
:1053B400202C19D02A00230001342F003240E4B2FB
:1053C4006D00002AF4D0524697654A465B085B009C
:1053D40022409B185B01434418009B4600F01EFCCE
:1053E400002808D1BE43E3D105B0F0BCBB46B246A9
:1053F400A946A046F0BD5B46E0219A78DB8A01A865
:1054040083600023C900018001210271437100F00F
:1054140025FC584600F0A0FBE4E7C046000011500C
:1054240000301150782000209823F0B5C646C84AB1
:1054340000B5D55880232E009B02102484B01E4052
:105444001D4274D0C34BC44C9A6AC44B00261A60E4
:105454003B23E35C022B00D14FE17B23E35C022B73
:1054640000D1F3E0BB23E35C022B00D1FAE0FB2381
:10547400E35C022B00D101E13C23FF33E35C022B0C
:1054840000D12DE17C23FF33E35C022B00D10EE13C
:10549400BC23FF33E35C022B00D13FE1FC23FF3349
:1054A400E35C022B00D1F5E0AD4BE35C022B00D1B1
:1054B40074E1AC4BE35C022B00D105E1AA4BE35C45
:1054C400022B00D175E1A94BE35C022B00D132E140
:1054D400A74BE35C022B00D1A0E1A64BE35C022BBB
:1054E40000D171E1A44BE35C022B00D1A1E1A34BF9
:1054F400E35C022B00D17FE1002E08D1A04B1B7886
:10550400002B04D180219F4A90338902D150C022BC
:1055140069468F4B92009B6C80265B058A805B0DED
:10552400012101A8029300F099FB974CB602EB0607
:1055340000D57FE080235B021D4231D01E4301234E
:1055440002249846844FBB7E002B14D000F090FCBC
:10555400012800D972E0C02200213800920100F035
:1055640001FB380000F0F8FA00F082FC012802D9AF
:10557400844B5C661C664346FB702037012C22D1A9
:10558400C0236A46DB009380804A02AB03CA03C38C
:10559400012101A800F062FB80227A4B92021A6575
:1055A40080235B011D4210D18023DB011D4223D1E6
:1055B40080231B021D422FD1AE4200D0C0E104B0B3
:1055C40080BCB846F0BD0124BDE700241E43604BF7
:1055D4001C60FFF7A5FE80236A465B00938014726B
:1055E400012101A800F03AFB8022664B12031A65E0
:1055F4008023DB011D42DBD01E4380236A46DB008F
:105604009380012101A800F029FB10225D4B1A654B
:1056140080231B021D42CFD01E43A0236A46DB0019
:105624009380012101A800F019FB8022554B12013F
:105634001A65C1E7FFF7A8FE26007BE7544B444AEE
:105644001C66536E2340A342FBD184E77833E75CA6
:10565400002F00D106E70233E25C002A00D00DE1FE
:105664003E00FFE6B833E75C002F00D1FFE60233CB
:10567400E25C002A00D0F9E03E00F8E6F833E75C8B
:10568400002F00D1F8E60233E25C002A00D041E1A9
:105694003E00F1E6F933FF33E75C002F00D103E766
:1056A4000233E25C002A00D02BE13E00FCE67933B1
:1056B400FF33E75C002F00D1EAE60233E25C002A04
:1056C40000D015E13E00E3E6324BE75C002F00D149
:1056D400F4E60233E25C002A00D001E13E00EDE68C
:1056E4003933FF33E75C002F00D1CBE60233E25CB1
:1056F400002A00D0EBE03E00C4E63833E65C002E1E
:1057040000D1AAE60233E25C002A00D1A5E620001B
:1057140000222030E25400F04DFA9EE6B933FF3304
:10572400E75C002F00D1B9E60233E25C002A00D026
:10573400C4E03E00B2E6184BE75C002F00D1C7E698
:105744000233E25C002A00D0B0E03E00C0E6C0466E
:105754000000115000400540782000206C200020FB
:105764003B0200007B020000BB020000FB020000C1
:105774003B0300007B030000BB030000FB030000AD
:10578400A12400200030115010000200000010502D
:10579400002011507A020000FA0200006B4BE75C13
:1057A400002F00D185E60233E25C002A76D13E0068
:1057B4007FE6674BE75C002F00D184E60233E25CAE
:1057C400002A63D13E007EE6624BE75C002F00D1E5
:1057D40088E60233E25C002A00D0A3E05E4BE35C7F
:1057E400022B30D15D4BE35C002B27D15C4BE35C97
:1057F400022B00D08BE63E005A4BE35C002B00D119
:105804007AE6FF239B00E25C002A00D17FE60022B7
:10581400E2541C3BE01800F0CDF978E6524BE75C0B
:10582400002F00D159E60233E25C002A16D13E0073
:1058340053E64A4BE35C002B00D158E6EF239B0070
:10584400E25C002A75D1464BE35C022B00D05EE695
:10585400444BE35C002B00D159E6D2E70022E2542A
:105864001C3BE01800F0A6F93E0036E620000022BA
:10587400A030E2543E0000F09DF9F8E5200000223B
:105884006030E2543E0000F095F9EBE50022E2546A
:105894001C3BE01800F08EF93E0014E60022E254AE
:1058A4001C3BE01800F086F93E0002E60022E254B8
:1058B4001C3BE01800F07EF93E0009E620000022BF
:1058C400A130FF30E2543E0000F074F9E6E5200018
:1058D40000222130FF30E2543E0000F06BF9D1E5A4
:1058E4000022E2541C3BE01800F064F93E00E5E5B8
:1058F400200000226130FF30E2543E0000F05AF9EB
:10590400C6E520000022E130FF30E2543E0000F002
:1059140051F9C9E520000022E030E2543E0000F0D5
:1059240049F9A9E50022E2541C3BE01800F042F9D1
:1059340054E70022E2541C3BE01800F03BF982E7F4
:1059440031000A48694000F083FAC0463A02000078
:10595400BA0200007A030000BB030000BA0300008F
:10596400FB030000FA0300003A0300006C4A001035
:10597400F0B5C64600B50200838A008B8C46011C34
:10598400984200D9191CD47880252000461EB041C5
:1059940089B2ED000D434003284301256C405B1A96
:1059A400D47054789BB29382002C31D16446D5686C
:1059B400A4014E1E2D19B0461469002923D0062EC9
:1059C40032D92B0023439B072ED1631CEB1A022BE5
:1059D4002AD900238F08BF00E658EE5004339F42B3
:1059E400FAD14346ED19DB1BE419B94209D02678F4
:1059F4002E70002B05D066786E70012B01D0A37831
:105A0400AB701469938A64181461802212021043E3
:105A1400002B02D18023DB0118436346002B00D006
:105A2400000480BCB846F0BD0023E65CEE540133AC
:105A34009942FAD1E5E7C0468368F0B51A680400D4
:105A4400002900D0120C63789205900D002B08D128
:105A5400E38AC318E382238B834201D90023A38200
:105A6400F0BDE368890125695E18471E002822D02D
:105A7400062F26D901315B18EB1A022B21D92B00F2
:105A840033439B071DD10023120E9200F158E950B5
:105A940004339A42FAD1BF1AAD18B618904209D00D
:105AA40032782A70002F05D072786A70012F01D0E5
:105AB400B278AA702569E38A2D18C318E382256198
:105AC400C9E70022B35CAB5401329042FAD1256994
:105AD400F1E7C04610B50400836800211B68FFF796
:105AE400ABFF63681B685B0002D5238B834200D045
:105AF40010BD01212000FFF79FFFF9E7084A0300CA
:105B0400126C0020920703D49A78D209012A00D09B
:105B14007047D87E023843425841C0B2F8E7C046C5
:105B24000000115010B5FFF7E9FF00280CD0074919
:105B3400074B8C46074A9B6A126863449B1A0020F1
:105B4400C6229A424041C0B210BDC046E0FCFFFFED
:105B5400004005406C2000200023837643610361EC
:105B64007047C04610B58368002901D01C682140E5
:105B7400002A12D08024E400114322420DD01A6876
:105B840022420CD1084A0A401A60084A126C920751
:105B940003D40C23033BFDD28368196010BD8178C4
:105BA400034800F055F9C046FFFBFFFF0000115009
:105BB400804A0010436870B50021802504001E68E7
:105BC400FFF7D6FE124B6D011A6C0543A3789207BA
:105BD4000ED55B060ED00F4B1E4080239B0533432E
:105BE40062680021136020002A00FFF7BBFF70BD2C
:105BF400DB09F0D0A38A002BEDD001212000FFF7B0
:105C0400B7FEA023044ADB05324005431343E7E70C
:105C140000001150FFFFFFAFFFFFFFDF70B5857E6F
:105C24000400002D14D0FFF755FFA38A002B01D1E7
:105C3400280070BD2000FFF775FF002803D0012362
:105C440000252377F4E72000FFF7B4FF0025EFE7F2
:105C54008178014800F0FCF8A04A0010F0B5CE4667
:105C6400474680B5437805000E0085B0062B08D85A
:105C74006B4A9B00D3589F466A4A13780133DBB2C0
:105C84001370694B1C686269EFF3108172B6136874
:105C9400002BFCD0BFF35F8FA1612000290000F02E
:105CA400F7F86269A369BFF35F8F0021116083F382
:105CB4001088002804D105B0C0BCB946B046F0BD78
:105CC40032006978287800F0EBF8F4E70121574BAB
:105CD4001A788A431A701A7801318A431A7000229A
:105CE4005A701A7802318A431A70CAE7504B514FDE
:105CF4009946514B002498463A7810E043461B6875
:105D040061015B18002B06D0DB69002B03D06968A6
:105D1400287898473A780134E4B2944217D8A242DA
:105D2400ECD8A31A5B014B44EEE7404B1A78D20738
:105D3400C1D504211A780A431A70A2E73B4B1A789A
:105D4400D207B8D504211A788A431A7099E7374FD5
:105D54003B785B072BD504223B78002193433B70AF
:105D64006B460632981D00F0A3F82B7801AC237023
:105D7400052363702C4B1B6898465A69EFF3108116
:105D840072B61368002BFCD0BFF35F8F43464046C6
:105D94009961210000F07CF843465A699B69BFF37E
:105DA4005F8F0021116083F31088002831D1FB78C4
:105DB400DB0700D47FE76B460A220021981D00F020
:105DC40077F82B7801AC2370032363706B686360EE
:105DD400154B1D686A69EFF3108172B61368002BC6
:105DE400FCD0BFF35F8FA9612800210000F050F8B8
:105DF4006A69AB69BFF35F8F0021116083F3108878
:105E0400002800D157E732006178207800F048F884
:105E140051E732006178207800F042F8C7E7C046C5
:105E2400084E0010A2240020741E00201C1E002016
:105E3400244E0010A0240020AC1C00207047C04653
:105E440001B40248844601BC604700BF71140010CD
:105E540001B40248844601BC604700BF110A001027
:105E640001B40248844601BC604700BFA11500107C
:105E740001B40248844601BC604700BF050A001013
:105E840001B40248844601BC604700BF752000107D
:105E940001B40248844601BC604700BFC539001004
:105EA40001B40248844601BC604700BF29280010A1
:105EB40001B40248844601BC604700BF6921001058
:105EC400204D00109C490010AC490010BC49001042
:105ED40010000000000000000000010000000000AD
:105EE40000000000000002000000000000000000AC
:105EF4000000030000000000000000000000FF009C
:105F04000000000001B5486801318E460047704624
:105F140009380149884701BDF50D00100000000053
:105F2400000000000000000000000000000000006D
:105F3400081600200000000000000000000000001F
:105F4400503300004C33000054330000523300003F
:105F54004D5300004D43000053340000433400000F
:105F6400781E002010000C0000000000000000005B
:105F7400000000000000000000000000FF0000001E
:105F8400A81000200000000000000000A819002054
:105F9400101A0020781A0020000000000000000001
:105FA40000000000000000000000000000000000ED
:105FB40000000000000000000000000000000000DD
:105FC40000000000000000000000000000000000CD
:105FD40000000000000000000000000000000000BD
:105FE40000000000000000000000000000000000AD
:105FF400000000000000000000000000000000009D
:10600400000000000000000000000000000000008C
:10601400000000000000000000000000000000007C
:1060240001000000000000000E33CDAB34126DE619
:10603400ECDE05000B000000000000000000000082
:10604400000000000000000000000000000000004C
:10605400000000000000000000000000000000003C
:10606400000000000000000000000000000000002C
:10607400000000000000000000000000000000001C
:10608400000000000000000000000000000000000C
:1060940000000000000000000000000000000000FC
:1060A40000000000000000000000000000000000EC
:1060B40000000000000000000000000000000000DC
:1060C4000000000000000000FFFFFFFF00000200CE
:1060D4000000000000000000F0110020F01100207A
:1060E400F8110020F81100200012002000120020F6
:1060F40008120020081200201012002010120020A4
:106104001812002018120020201200202012002053
:106114002812002028120020301200203012002003
:1061240038120020381200204012002040120020B3
:106134004812002048120020501200205012002063
:106144005812002058120020601200206012002013
:1061540068120020681200207012002070120020C3
:106164007812002078120020801200208012002073
:106174008812002088120020901200209012002023
:106184009812002098120020A0120020A0120020D3
:10619400A8120020A8120020B0120020B012002083
:1061A400B8120020B8120020C0120020C012002033
:1061B400C8120020C8120020D0120020D0120020E3
:1061C400D8120020D8120020E0120020E012002093
:1061D400E8120020E8120020F0120020F012002043
:1061E400F8120020F81200200013002000130020F1
:1061F400081300200813002010130020101300209F
:10620400181300201813002020130020201300204E
:1062140028130020281300203013002030130020FE
:1062240038130020381300204013002040130020AE
:10623400481300204813002050130020501300205E
:10624400581300205813002060130020601300200E
:1062540068130020681300207013002070130020BE
:10626400781300207813002080130020801300206E
:10627400881300208813002090130020901300201E
:106284009813002098130020A0130020A0130020CE
:10629400A8130020A8130020B0130020B01300207E
:1062A400B8130020B8130020C0130020C01300202E
:1062B400C8130020C8130020D0130020D0130020DE
:1062C400D8130020D8130020E0130020E01300208E
:1062D400E8130020E8130020F0130020F01300203E
:1062E400F8130020F81300200014002000140020EC
:1062F400081400200814002010140020101400209A
:106304001814002018140020201400202014002049
:1063140028140020281400203014002030140020F9
:1063240038140020381400204014002040140020A9
:106334004814002048140020501400205014002059
:106344005814002058140020601400206014002009
:1063540068140020681400207014002070140020B9
:106364007814002078140020801400208014002069
:106374008814002088140020901400209014002019
:106384009814002098140020A0140020A0140020C9
:10639400A8140020A8140020B0140020B014002079
:1063A400B8140020B8140020C0140020C014002029
:1063B400C8140020C8140020D0140020D0140020D9
:1063C400D8140020D8140020E0140020E014002089
:1063D400E8140020E8140020F0140020F014002039
:1063E400F8140020F81400200015002000150020E7
:1063F4000815002008150020101500201015002095
:106404001815002018150020201500202015002044
:1064140028150020281500203015002030150020F4
:1064240038150020381500204015002040150020A4
:106434004815002048150020501500205015002054
:106444005815002058150020601500206015002004
:1064540068150020681500207015002070150020B4
:106464007815002078150020801500208015002064
:106474008815002088150020901500209015002014
:106484009815002098150020A0150020A0150020C4
:10649400A8150020A8150020B0150020B015002074
:1064A400B8150020B8150020C0150020C015002024
:1064B400C8150020C8150020D0150020D0150020D4
:1064C400D8150020D8150020E0150020E015002084
:1064D400E8150020E815002000000000000000007E
:0864E4000000000000000000B0
:04000005100001E9FD
:00000001FF
